:020000040000FA
:020000000528D1
:080008007228031383129F010B
:10001000831606309F0037308500FF30860087004A
:1000200088008900803081008312083085008B139E
:100030001C2021182E2018282110051A2D286C208C
:100040001830A0006E20A20DA30DA40D2214051ED1
:100050002210A00B22286E20211408002208FF3A4B
:100060008316860083122308FF3A831687008312C3
:1000700024087F39FF3A8316880083125E208601A8
:1000800087018801A41F4B282208860023088700C7
:1000900024087F3988005E2085116E20851583161F
:1000A000FF30860087008800831208000530A50015
:1000B000000000000000A50B5A2808003C3057281B
:1000C000A7000A30A6006428652800005E20A60B61
:1000D0006528A70B612808000230602804306028DA
:1000E00064306028F0000308F100831203130B1D35
:1000F00005280B1181017C2871088300F00E700E19
:020100000900F4
:02400E00323F3F
:1042000043006F0070007900720069006700680069
:1042100074002000280043002900200032003000F4
:10422000310030002D003200300031003800200015
:104230006200790020004D002E00590061006D00E1
:0A42400061006D006F0074006F0054
:00000001FF
